:1000000088C0B0C0AFC0AEC0ADC0B1C0ABC0AAC0A8
:10001000A9C0A8C0A7C0A6C0A5C0A4C0A3C074455D
:1000200079467D47824887498B60906194629963E5
:100030009D64A265A766AB67B068B469B980BE81EC
:10004000C282C783CB84D084D484FF210000000007
:100050000000000000000000000023456C98C9FF6C
:10006000040714233764A0FFFFFFFFFFFFFFFFFF1C
:10007000FFFFFF00000000000000000023405F7A47
:10008000B4FFFFFFFFFFFF001400081400080E1468
:100090000004080E14000305080E14000305080AE6
:1000A0000E14000305080A0E1014000305080A0EBA
:1000B0001012140008000E00080E0004080E0003C1
:1000C00005080E000305080A0E0004080E101400AF
:1000D000F3F404080E10121400080A0C0E0F10128C
:1000E0001400080EEE1400020304050004140004BA
:1000F0000E1400040810140004080F111400EEED93
:10010000ECEB140E08040004080E00EBECEDEEF32B
:10011000F41411241FBECFE5D2E0DEBFCDBF20E036
:10012000A0E6B0E001C01D92A638B207E1F7E1E613
:10013000F0E085E5808781E08383148212828683E4
:100140001182ACE6B0E08EEF15968C9315978DEF8B
:1001500017968C938BE0818788E58287612C712CC0
:10016000B8D0B2C24DCF1BBC19BC18BC08951895AD
:1001700025B7277E25BF29B7226029BF21E022BFEE
:10018000019728F020E188952150E9F7F9CF0895EB
:1001900088EE93E0EDCF81EA87B986EC86B9369A8E
:1001A0000895369A3699FECF85B10895CF93C72D1D
:1001B00081E0870D8F73782E662D90E077D26FEFF8
:1001C0008C2F90E0CF9172C2FF920F931F93CF9329
:1001D000DF93F82E0BE610E0C5E7D0E081E0F812DF
:1001E00005C0F8016081CE0161D204C0CE0156D2B3
:1001F000F8018083015011092196CF37D10571F79D
:10020000DF91CF911F910F91FF900895CFDF81E093
:10021000DBCF811101C0A7CF815090E0FC01E45BEE
:10022000FF4FE491EBBDFC01E05AFF4FE491E9BDC3
:10023000FC01EC58FF4F849188BD08950F931F93E4
:10024000CF93C82F8B01CC2359F085E0E2DFC801A2
:100250008FDF89DFC8018CDFC8018ADFC150F3CF8F
:10026000CF911F910F910895EF92FF920F931F93DB
:10027000CF93C8E0E82EF12C062F10E084E1C9DF0F
:10028000C70176DF70DFC80173DFC150B9F7CF91C6
:100290001F910F91FF90EF9008951F93CF93DF93DD
:1002A0008FEA87B986EC86B910E1C0E0D0E085E03E
:1002B00090E05EDF76DFC80FD11D1150C1F7CE018F
:1002C00024E0969587952A95E1F7DF91CF911F91CC
:1002D000089583EA87B986EC86B93699FECF369AB7
:1002E0003699FECFC5B18FE384BBBB9AC39AB99A46
:1002F000B89ABC9A81E08ABD83BF9AB590629ABDD4
:100300009AB590689ABD9FEF9DBD80BF80E68CBD79
:1003100097B328B3892F90E0809590958B7F822B9F
:1003200088BB85B7806285BF789487E790E0B6D1B7
:10033000853511F06BDF11C0712C872D90E0AED1A7
:10034000682E8F3F19F080E03FDF07C0872D91E0D6
:10035000970D792E803488F3F6CF80916A00009152
:100360006400F090650010916200112319F0F12CE7
:1003700000E088E18F5F90E040E050E068E870E0E6
:10038000882379F09B012F5F3F4FF9013197E4916A
:10039000EE2319F0922F961BF6CF8150AB01B901D5
:1003A000EFCF892F602F70E0A92FB0E0E82FF0E0A9
:1003B000FF2021F09D012E1B3F0B05C09F01215006
:1003C0003109260F371F3197E40FF51FE4902B58A2
:1003D0003F4FF901E082815049F7900F9093600000
:1003E000002371F0FF2029F0292F30E0215031093E
:1003F00002C020E030E0F901EB58FF4F81E080833C
:1004000087E0890F282F2150E22FE91BF0E0E55FFC
:10041000FE4FE491A22FB0E0AB58BF4FEC932913ED
:10042000F2CFE82FF0E0EC58FF4F21E0409175004B
:100430003081431320E0821B282F80938500862D76
:10044000853F70F5C93F60F08F5F682E891708F00F
:10045000612C809186008F5F8F718093860020C011
:1004600010928600C33DB0F030916700332311F045
:10047000112331F08F5F682E891790F0612C10C026
:100480006916E1F3662019F08150682E09C02150E9
:10049000622E06C01111F2CF80916300882371F3A0
:1004A00085DE79DEC62DC53F28F4D0E0CB58DF4F7E
:1004B000C881DC2F10E000E0EE24E39480918600F8
:1004C000803190F165DE10928600C2E6D0E0C12C4A
:1004D000D12C81E08C0DFFEFCF1ADF0A98819F3F6E
:1004E00031F4219688E0C816D10499F718C06DE55B
:1004F00070E0A4DEF601E459FF4F608088818E250C
:10050000888384DE6FE070E080E298DE88818E254B
:1005100088837CDE3DDE80916200882311F3612CAC
:10052000C0917500DC2F8EC0CE3E19F463E481E2E9
:1005300004C0CD3E21F468E284E196DE83C0CC3E67
:1005400011F469E203C0CB3E19F462E581E0F5CF16
:10055000C33F41F484E15DDE8AE090E009DE88E09B
:1005600058DE3DC0C43F59F584E690E001DE13DE5D
:1005700018DE90E0292F30E0F901E25EFF4FE491B0
:10058000E81710F49E5FF6CFF901E15EFF4FF4909B
:100590006DE770E08F2D8295869587704FDE8EEE29
:1005A00092E0E6DD65E070E081E048DE85E694E01B
:1005B000DFDD6DE770E08F2D8F7140DE0FC0CE3F25
:1005C00081F4612CF12CF0926A0020DE6AEF70E079
:1005D00081E034DEF39498E1F912F5CFD9DDD8DD6E
:1005E00031C0CD3F91F4612C8FEF80936B000EDE14
:1005F00085E00FDECDDDCCDD84E10BDE4EDE8093C9
:100600006B0004DEC5DDC4DDF9CF8D2F02DE45DED3
:1006100020916B00821738F00F5F093078F0D330EB
:1006200068F0D1500AC090E030E0225031098217C2
:1006300093071CF4DC1708F4DF5F00E0ACDD84EF07
:1006400091E096DD10928600ACDD823890F41F5F59
:10065000183008F433CFD53120F010E0DAE0CAE0EA
:100660002DCFD23040F08D2F86958695D695D80F18
:10067000CD2F10E023CF77DD85B7877E806185BFE2
:10068000F89485B7846885BF8B7F85BF85B7806206
:1006900085BF889585B78F7D85BFEACFE199FECF6D
:1006A0009FBB8EBBE09A99278DB30895262FE199C1
:1006B000FECF1CBA9FBB8EBB2DBB0FB6F894E29A3F
:0C06C000E19A0FBE01960895F894FFCF58
:00000001FF
